:1000000002095D7DA37C08ED1D70011C144C70F786
:0F001000EF1F70011E144E70EA22AE070209693D
:100023000208AAE518240CF8E60518227809300717
:1000330002780CE475F0011205320203822000EB12
:100043007F2ED2008018EF540F2490D43440D4FF75
:1000530030040BEF24BFB41A0050032461FFE519E9
:1000630060021519051CE51C7002051B30070D788D
:1000730009E475F001120532EF0204EA02001A7472
:1000830003D2078003E4C207F5188B098A0A890B98
:10009300E4F519F51BF51CE51960077F20120061D3
:1000A30080F5751AFFC201C200C202C203C205C2B3
:1000B30006C20812002FFF700D3007057F001200E3
:1000C30072AF1CAE1B22B4255FC2D5C20412002F2F
:1000D300FF24D0B40A00501A75F00A781930D505F8
:1000E30008B6FF0106C6A426F620D5047002D20383
:1000F30080D924CFB41A00EF5004C2E5D20402021F
:1001030072D20180C6D20080C0D20280BCD2D58018
:10011300BAD20580B47F201200612002077401B5B2
:10012300190040F1120026FF12006102009AD20862
:10013300D2068095120026FB120026FA120026F939
:100143004A4B700679437A037BFF20022EE5196040
:100153002A7E008E8275830012039B60060EEE6575
:100163001A70F0C2D5EBC0E0EAC0E0E9C0E0EE12DD
:1001730002B9D0E0F9D0E0FAD0E0FB120382FF60CD
:10018300AAEBC0E0EAC0E0E9C0E0120061D0E024DD
:1001930001F9D0E03400FAD0E0FBE51A0460DCD5C5
:1001A3001AD980877BFF7A0279B5D202809C7910B5
:1001B30080027908C206C2088008D2D5790A800471
:1001C300790AC2D5E51A047002F51AE4FAFDFEFFB6
:1001D300120026FC7B08200113120026FD7B103041
:1001E300000A120026FE120026FF7B20EC3382D584
:1001F30092D55013C3E43000069FFFE49EFEE42033
:1002030001039DFDE49CFCE4CBF8C201EC700CCF30
:10021300CECDCCE824F8F870F38017C3EF33FFEEAC
:1002230033FEED33FDEC33FCEB33FB994002FB0F64
:10023300D8E9EB300105F8D0E0C448B201C0E00AC8
:10024300EC4D4E4F78207B0070C2EAB51A0040BCDB
:10025300C0E01202BBD0F0D0E0200104C4C0E0C46F
:10026300B201C0F012004AD0F0D5F0EB02009A12AE
:10027300054201375301B15801084C01044201B54D
:100283004F01BD4401BD49011D4301C35501A746AB
:1002930001A74501A747036350010C2D01102E014F
:1002A300332B011423013120034C2A00CC480000D6
:1002B300012B3F3F3F00790AA2D5200314300509E3
:1002C300B910020404B9080104A2D52006025001A2
:1002D300042002689202B519005034C0E07F203038
:1002E30003197F30A20272067205500F120312C265
:1002F30002C206C205C2087F30800F300503E9C081
:10030300E0120061300503D0E0F9D0E0B519CC303C
:1003130005177F30B9100C1200617F583004077F36
:10032300788003B908031200613002057F2D0200B3
:10033300617F202008F87F2B2006F322920280CFD2
:10034300286E756C6C2900D2011200263001F8C2A8
:1003530001781930D50108F60200CC2D50434958D5
:100363001200262403B405004001E490035E9312B7
:100373000052743A120052D2037519040201B1BB40
:10038300010689828A83E0225002E722BBFE02E350
:100393002289828A83E49322BB010CE58229F582B8
:1003A300E5833AF583E0225006E92582F8E622BB8D
:1003B300FE06E92582F8E222E58229F582E5833A01
:1003C300F583E4932275F008758200EF2FFFEE3377
:1003D300FECD33CDCC33CCC58233C5829BED9AECB5
:1003E30099E58298400CF582EE9BFEED9AFDEC991F
:1003F300FC0FD5F0D6E4CEFBE4CDFAE4CCF9A88229
:1004030022B800C1B90059BA002DEC8BF084CFCECD
:10041300CDFCE5F0CBF97818EF2FFFEE33FEED338B
:10042300FDEC33FCEB33FB10D703994004EB99FB52
:100433000FD8E5E4F9FA227818EF2FFFEE33FEED3B
:1004430033FDEC33FCC933C910D7059BE99A400748
:10045300EC9BFCE99AF90FD8E0E4C9FAE4CCFB225F
:1004630075F010EF2FFFEE33FEED33FDCC33CCC828
:1004730033C810D7079BEC9AE899400AED9BFDEC33
:100483009AFCE899F80FD5F0DAE4CDFBE4CCFAE472
:10049300C8F922EB9FF5F0EA9E42F0E99D42F0E8AD
:1004A3009C45F022E8600FECC313FCED13FDEE1343
:1004B300FEEF13FFD8F122BB010DE58229F582E59A
:1004C300833AF5830205095007E92582F80204FC03
:1004D300BBFE07E92582F8020515E58229F582E5C9
:1004E300833AF583020522BB010689828A83F022BF
:1004F3005002F722BBFE01F322E6FB08E6F908E609
:10050300FA08E6CBF822E0F8A3E0F9A3E0FAA3E0C7
:10051300FB22E2FB08E2F908E2FA08E2CBF822E464
:1005230093F8740193F9740293FA740393FB22FA18
:10053300E6FB0808E6F925F0F618E6CA3AF622D0F3
:1005430083D082F8E4937012740193700DA3A39384
:10055300F8740193F5828883E4737402936860EFFF
:10056300A3A3A380DF8B128A138914EF64016003B2
:100573000206D1752201F523F524F525F526F52785
:10058300F528FFEFC3948074809480500F74802FFC
:10059300F582E43400F583E4F00F80E7E4FFEFC372
:1005A300948074809480500F74002FF582E434009B
:1005B300F583E4F00F80E7AB12AA13A914120382A8
:1005C300FFE598543F4FF598EF64C06008EF64402F
:1005D30060030206809000021204BA7F007E607DF1
:1005E300547C001204048F188E178D168C15E4FFAB
:1005F300FE7D01FCAB18AA17A916A815C312049611
:1006030040037FFF22C3E49518F518E49517F51707
:1006130074019516F516E49515F515AB12AA13A9F1
:100623001490000112039B64027026538EEF438ED5
:1006330001538EF7438E04AF18AE17AD16AC157881
:10064300081204A78FD68518D753AFFB438E1080AB
:1006530066C28E538EFE5389BF5389CF438E40AFFC
:1006630018AE17AD16AC1578081204A78F8D851830
:100673008BC2AB5389BF538FFDD28E803AAB12AA84
:1006830013A914120382FF7E007014900008120352
:100693009B64017005438E20801D538EDF8018EF0D
:1006A30064804E701290000812039B64017005432E
:1006B3008780800353877FAB12AA13A91490000786
:1006C30012039B7004C29C8002D29C7F00227FFF96
:1006D30022EFD3940F7480948040028063E4F5BDCD
:1006E300F5BEE5BC54F044404FF5BC00000000E407
:1006F300FDEDC394FA748094805045E5BC30E53D2C
:1007030053BCDFE5DEAFBD30E50EEFFEACBEECFB68
:10071300EEF509EBF50A80207509008F0AE5BEC4E2
:10072300540FFBE50AC4F8540FC868FFE509C45425
:10073300F048F509EF4BF50AAE09AF0A220D80B177
:100743007E107F002290000112039BFFE5DE54F030
:100753004FF5DE90000212039BC43354E0FFE5DE45
:1007630054DF4FF5DE120382D3941F7480948050BC
:100773003D90000312039BFFD39401748094805037
:100783002D90000412039BFED39403748094805035
:100793001D43BA80EEC43354E0FEEFC43333335405
:1007A300804EFF1203824F90FEA8F053BA7F2212AD
:1007B300093D1208F512091CD2AF7BFF7A09797340
:1007C300120088E4F508C3E50894107480948050FF
:1007D300317FC87E00120003AF081206D47BFF7A74
:1007E30009799585080C8E0D8F0E120088E5085443
:1007F30007640770097BFF7A0979A312008805084B
:1008030080C47BFF7A0979A312008880B6EFFBD3FB
:100813009401748094805009EB7004C2AD8002D2BD
:10082300ADEDFF7E00D39403748094805029EF7064
:100833000553B7DFC2BDEF64014E700553B7DFD276
:10084300BDEF64024E700543B720C2BDEF64034E93
:10085300700543B720D2BD7F0022EFFBD394017410
:100863008094805009EB7004C2AC8002D2ACEDFFDF
:100873007E00D39403748094805029EF700553B79E
:10088300EFC2BCEF64014E700553B7EFD2BCEF6407
:10089300024E700543B710C2BCEF64034E700543AC
:1008A300B710D2BC7F0022C0E0C083C082C0D07525
:1008B300D000C007309828C298E5287022C3E526E7
:1008C3009480748094804003752600AF26052674B7
:1008D300002FF582E43400F583E599F075270530A0
:1008E3009905C299752500D007D0D0D082D083D086
:1008F300E032750940750A01750E00750DC2750C5D
:1009030001750B007510017B007A0079097F0112D4
:1009130005687D017F0102085D75091FE4F50C750B
:100923000D01F50A750B01FB7A0079091207487F5F
:1009330001120950E4FDFF02081043937F53948092
:100943007591FF75920053B1FC53B2FC22EF640121
:10095300700443BC802253BC7F22787FE4F6D8FD29
:100963007581280207B28F99752501E52570FC2250
:100973005354433820414420746F2055415254202E
:10098300546573742050726F6772616D6D65210DCC
:100993000A00414425303262643D2530346420002E
:0309A3000D0A003A
:00000001FF
